:020000040000FA
:020000000428D2
:0800080007309F00831603136B
:10001000DF30850001308600073081008312031332
:10002000D501851B5514D301203084005308840763
:1000300038205518FF3A800004168000D30A531E5A
:1000400014283030840000305518FF30D400800070
:10005000203084000618302805080F39203E84001F
:100060000412051F04160008051E540986002A28DC
:10007000831603139B001C141A0883120313080031
:02400E00703F01
:104200007E000C009E00B6000E00FA00CC00DA0022
:10421000E200F200B000BC00FE00DE00F800EE009C
:104220002000420069006E006100720079002000E9
:1042300074006F00200037002D00730065006700D8
:104240006D0065006E00740020006400650063006E
:104250006F006400650072002000200056003100ED
:104260002E0030002E0031002000200032003400EB
:104270002F00300031002F003200300031003500B7
:1042800020002000700069006300700072006F0061
:104290006A0065006300740073002E006F007200F6
:0A42A00067002E0075006B0020007F
:00000001FF
